:1000000061C05AC17AC079C078C077C076C075C067
:1000100074C073C072C071C070C06FC06EC06DC05C
:100020006CC06BC06AC005010905A1010901A100EE
:100030000930093115FF2501750295028102C005BD
:10004000091901292415002501750195248102C093
:10005000040309042403700075006C006B006F003A
:100060006D0061006E00640079002E006100740074
:1000700068002E00630078001803530074006100CC
:1000800072006B006100640072006F006900640020
:100090001201100100000008424231170001010264
:1000A0000001090222000101008032090400000160
:1000B00003000000092101010001222A0007058137
:1000C0000308000A11241FBECFE5D4E0DEBFCDBF78
:1000D00010E0A0E6B0E0E6EAF7E002C005900D927D
:1000E000A436B107D9F710E0A4E6B0E001C01D9234
:1000F000A23AB107E1F741D054C382CFFC0185E6B3
:1001000090E0909387008093860080818076803293
:1001100071F58181813011F485E00895893049F4C9
:1001200086819781019719F581E0809364008FEFB4
:100130000895823019F48AE690E013C08A3029F4D9
:10014000838180936A0080E00895833031F4838155
:10015000882369F41092600008958B3041F480E6A2
:1001600090E0909387008093860081E0089580E07E
:1001700008951092640081E00895EF92FF920F932A
:100180001F93CF93DF932FE088E190E00FB6F894B0
:10019000A89581BD0FBE21BDB0D1789417BA8FEF5D
:1001A00088BB14BA85BB84E083BF10E0C1E0D0E017
:1001B0005FEDF52E0FEFEE24E394A895ABD120E090
:1001C00030E0CE01022E02C0880F991F0A94E2F798
:1001D000809587BB88BB83B3F901EB59FF4F8095AE
:1001E0008F7380832F5F3F4F2530310551F7F7BA6A
:1001F000F8BA83B390E08095909546E0880F991FF8
:100200004A95E1F720916500282B2093650083B380
:1002100090E08095909534E0880F991F3A95E1F72A
:10022000807C20916600822B8093660083B390E0EF
:1002300080959095880F991F880F991F807C209139
:100240006700822B8093670007BB08BB8091770013
:1002500084FF04C085E690E065E081D208B600FE28
:10026000ACCFE8BE812F8F5F853010F01450A5CF42
:1002700010916A008091770084FF9FCF85E690E01F
:1002800065E06DD29ACFA82FB92F80E090E041E0D1
:1002900050EA609530E009C02D91822797958795A7
:1002A00010F084279527305EC8F36F5FA8F3089598
:1002B000EADF8D939D930895CF93CFB7CF93DF93CC
:1002C000C395859BE9F7859B0BC0859B09C0859BE2
:1002D00007C0859B05C0859B03C0859B01C08BC063
:1002E0006F93C0918500DD27C457DF4F2F9365E5DD
:1002F000859B03C02F916F91E6CF0F931F934F9370
:1003000020E040E15F9300B3047205FB27F93F93BF
:1003100050E03BE039C0147240642F77012F5F5FDB
:100320001EC0406810B314722F7752501FC0406433
:1003300000B32F770472D1F15F5F00C023C0406229
:1003400010B32F77147291F15F5F00C025C0047263
:100350001027515012F45D5F0000115027952C3F7B
:1003600010B3C8F614720127015027952C3FC8F628
:100370004227499300B3047210274F7311502795F9
:100380002C3FA8F64695469510B3147279F00127D4
:10039000015027952C3F98F66B5A60F3315000B30B
:1003A000B0F600C010E41ABF002719C03B503195C9
:1003B000C31BD04010E41ABF0881033C09F10B3481
:1003C000F9F0209183001981110F1213EDCF4A81AA
:1003D000441F093651F10D3211F0013E29F7009307
:1003E0008A003F915F914F911F910F912F916F91D3
:1003F000CAB7C6FD65CFDF91CF91CFBFCF9118951A
:1004000020918A00222369F310918800112391F52D
:10041000343092F13093880020938400109185004D
:100420003BE0311B3093850027C0009188000130EC
:100430000CF50AE54F7049F43091610034FD1DC0A0
:1004400000936100CCE6D0E01CC03091770034FD11
:1004500014C000937700C8E7D0E013C0052710E070
:1004600000C0000002BB1AC0052710E0221F1DC0FB
:1004700010E021C04AE502C032ED432FC4E1D0E0D4
:1004800032E011B31462959A02B311BB54E220E832
:1004900065E320FF052702BB279517951C3FF0F663
:1004A0006695B8F7B1F720FF052702BB279517958A
:1004B0001C3FD0F62795179517FF052700001C3F16
:1004C00002BBB0F629913A9519F70B7D109189007E
:1004D000110FC651D04002BB11F01093830010E4FD
:1004E0001ABF006211B31B7D402F4B7D54E05A951B
:1004F000F1F702BB11BB42BB74CF85B7836085BFE8
:100500008BB780648BBF8BE4809378008AE58093FF
:10051000770008951F93CF93DF9360918800635015
:1005200067FDC2C080918500CCE0D0E0C81BD10936
:10053000C457DF4F809184008D3209F0A3C068302A
:1005400009F0B0C083EC80936C008AE58093610071
:1005500010926B008881807639F0CE01CFDD282F94
:100560008F3F09F47EC084C09A8110927500898102
:10057000882321F41092760022E06CC0853019F4B3
:100580009093890066C0863009F04FC08B8181301E
:1005900041F480E990E0909387008093860022E107
:1005A00040C0823041F482EA90E0909387008093CB
:1005B000860022E236C08330F9F48A81882341F430
:1005C00080E590E0909387008093860024E029C026
:1005D000813041F484E590E0909387008093860019
:1005E00024E21FC08230E1F488E790E09093870016
:1005F0008093860028E115C0813241F484EB90E0BD
:10060000909387008093860029E00BC0823241F4EA
:1006100086E290E090938700809386002AE201C0F2
:1006200020E080E480936B0023C0883021F421E037
:100630008BE890E011C0893019F490938B0009C0C9
:100640008A3011F421E006C08B3019F48BE48093DA
:10065000780020E085E790E0909387008093860003
:1006600007C0888187FD2E8180E880936B0006C0DB
:100670008F81882319F48E81821708F0822F80934E
:10068000620010C080916B0087FF0CC0CE0171DD4D
:100690008F3F21F48EE18093610004C0882311F024
:1006A00010926200109288008091610084FF49C01E
:1006B000809162008F3F09F444C0182F893008F000
:1006C00018E0811B8093620080916C0098E8892774
:1006D00080936C00112341F12091860030918700B6
:1006E00080916B0086FF0DC0ADE6B0E080E090E049
:1006F000F901E80FF91FE491ED9301961817C1F77E
:1007000008C0912FD901EDE6F0E08D9181939150D1
:10071000E1F71150812F90E01F5F0196820F931F28
:1007200090938700809386008DE690E0612FC0DD76
:10073000612F6C5F6C3019F08FEF809362006093D3
:10074000610094E180B3847231F49150D9F7109232
:10075000890010928300DF91CF911F9108951F931C
:10076000DC01162F8091770084FF07C0809178000C
:1007700098E889278093780003C08AE58093770002
:10078000912FE9E7F0E08D91819391501916DCF3F8
:1007900089E790E0612F8CDD1C5F109377001F913B
:0607A0000895F894FFCF5C
:0407A600015AFF00F5
:00000001FF
